 le

 Timestamp is 89eed5ef (reproducible build file hash)

 Preferred load address is 10000000

 Start         Length     Name                   Class
 0001:00000000 00002409H .text$mn                CODE
 0002:00000000 000000bcH .idata$5                DATA
 0002:000000bc 00000008H .00cfg                  DATA
 0002:000000c4 00000004H .CRT$XCA                DATA
 0002:000000c8 00000004H .CRT$XCZ                DATA
 0002:000000cc 00000004H .CRT$XIA                DATA
 0002:000000d0 00000004H .CRT$XIZ                DATA
 0002:000000d4 00000004H .CRT$XPA                DATA
 0002:000000d8 00000004H .CRT$XPZ                DATA
 0002:000000dc 00000004H .CRT$XTA                DATA
 0002:000000e0 00000008H .CRT$XTZ                DATA
 0002:000000e4 00000000H .gfids$y                DATA
 0002:000000e8 00000a98H .rdata                  DATA
 0002:00000b80 00000000H .rdata$CastGuardVftablesA DATA
 0002:00000b80 00000000H .rdata$CastGuardVftablesC DATA
 0002:00000b80 0000012cH .rdata$r                DATA
 0002:00000cac 00000004H .rdata$sxdata           DATA
 0002:00000cb0 0000005cH .rdata$voltmd           DATA
 0002:00000d0c 000002d0H .rdata$zzzdbg           DATA
 0002:00000fdc 00000004H .rtc$IAA                DATA
 0002:00000fe0 00000004H .rtc$IZZ                DATA
 0002:00000fe4 00000004H .rtc$TAA                DATA
 0002:00000fe8 00000008H .rtc$TZZ                DATA
 0002:00000ff0 00000120H .xdata$x                DATA
 0002:00001110 00000578H .edata                  DATA
 0002:00001688 00000050H .idata$2                DATA
 0002:000016d8 00000014H .idata$3                DATA
 0002:000016ec 000000bcH .idata$4                DATA
 0002:000017a8 00000416H .idata$6                DATA
 0003:00000000 00000018H .data                   DATA
 0003:00000018 00000060H .data$r                 DATA
 0003:00000078 00000018H .data$rs                DATA
 0003:00000090 00000484H .bss                    DATA
 0004:00000000 00000060H .rsrc$01                DATA
 0004:00000060 00000318H .rsrc$02                DATA

  Address         Publics by Value              Rva+Base       Lib:Object

 0000:00000000       ___AbsoluteZero            00000000     <absolute>
 0000:00000000       ___arm64x_extra_rfe_table  00000000     <absolute>
 0000:00000000       ___arm64x_extra_rfe_table_size 00000000     <absolute>
 0000:00000000       ___arm64x_native_entrypoint 00000000     <absolute>
 0000:00000000       ___arm64x_redirection_metadata 00000000     <absolute>
 0000:00000000       ___arm64x_redirection_metadata_count 00000000     <absolute>
 0000:00000000       ___dynamic_value_reloc_table 00000000     <absolute>
 0000:00000000       ___enclave_config          00000000     <absolute>
 0000:00000000       ___guard_check_icall_a64n_fptr 00000000     <absolute>
 0000:00000000       ___guard_eh_cont_count     00000000     <absolute>
 0000:00000000       ___guard_eh_cont_table     00000000     <absolute>
 0000:00000000       ___guard_fids_count        00000000     <absolute>
 0000:00000000       ___guard_fids_table        00000000     <absolute>
 0000:00000000       ___guard_iat_count         00000000     <absolute>
 0000:00000000       ___guard_iat_table         00000000     <absolute>
 0000:00000000       ___guard_longjmp_count     00000000     <absolute>
 0000:00000000       ___guard_longjmp_table     00000000     <absolute>
 0000:00000000       ___hybrid_auxiliary_delayload_iat 00000000     <absolute>
 0000:00000000       ___hybrid_auxiliary_delayload_iat_copy 00000000     <absolute>
 0000:00000000       ___hybrid_auxiliary_iat    00000000     <absolute>
 0000:00000000       ___hybrid_auxiliary_iat_copy 00000000     <absolute>
 0000:00000000       ___hybrid_code_map         00000000     <absolute>
 0000:00000000       ___hybrid_code_map_count   00000000     <absolute>
 0000:00000000       ___hybrid_image_info_bitfield 00000000     <absolute>
 0000:00000000       ___x64_code_ranges_to_entry_points 00000000     <absolute>
 0000:00000000       ___x64_code_ranges_to_entry_points_count 00000000     <absolute>
 0000:00000001       ___safe_se_handler_count   00000001     <absolute>
 0000:00000100       ___guard_flags             00000100     <absolute>
 0000:00000000       ___ImageBase               10000000     <linker-defined>
 0001:00000000       ?NewObject@JNIEnv_@@QAAPAV_jobject@@PAV_jclass@@PAU_jmethodID@@ZZ 10001000 f i Kernel32.obj
 0001:00000018       _Java_jdk_internal_org_jline_terminal_impl_jna_win_Kernel32Impl_FillConsoleOutputAttribute@28 10001018 f   Kernel32.obj
 0001:000000c3       _Java_jdk_internal_org_jline_terminal_impl_jna_win_Kernel32Impl_FillConsoleOutputCharacter@28 100010c3 f   Kernel32.obj
 0001:0000016e       _Java_jdk_internal_org_jline_terminal_impl_jna_win_Kernel32Impl_GetConsoleMode@16 1000116e f   Kernel32.obj
 0001:000001e0       _Java_jdk_internal_org_jline_terminal_impl_jna_win_Kernel32Impl_GetConsoleScreenBufferInfo@16 100011e0 f   Kernel32.obj
 0001:000003e4       _Java_jdk_internal_org_jline_terminal_impl_jna_win_Kernel32Impl_GetStdHandle@12 100013e4 f   Kernel32.obj
 0001:00000403       _Java_jdk_internal_org_jline_terminal_impl_jna_win_Kernel32Impl_ReadConsoleInput@24 10001403 f   Kernel32.obj
 0001:00000833       _Java_jdk_internal_org_jline_terminal_impl_jna_win_Kernel32Impl_ScrollConsoleScreenBuffer@28 10001833 f   Kernel32.obj
 0001:000009ae       _Java_jdk_internal_org_jline_terminal_impl_jna_win_Kernel32Impl_SetConsoleCursorPosition@16 100019ae f   Kernel32.obj
 0001:00000a38       _Java_jdk_internal_org_jline_terminal_impl_jna_win_Kernel32Impl_SetConsoleMode@16 10001a38 f   Kernel32.obj
 0001:00000a92       _Java_jdk_internal_org_jline_terminal_impl_jna_win_Kernel32Impl_SetConsoleTextAttribute@16 10001a92 f   Kernel32.obj
 0001:00000aec       _Java_jdk_internal_org_jline_terminal_impl_jna_win_Kernel32Impl_SetConsoleTitle@12 10001aec f   Kernel32.obj
 0001:00000b4e       _Java_jdk_internal_org_jline_terminal_impl_jna_win_Kernel32Impl_WaitForSingleObject@16 10001b4e f   Kernel32.obj
 0001:00000b7d       _Java_jdk_internal_org_jline_terminal_impl_jna_win_Kernel32Impl_WriteConsoleW@28 10001b7d f   Kernel32.obj
 0001:00000c42       _Java_jdk_internal_org_jline_terminal_impl_jna_win_Kernel32Impl_initIDs@8 10001c42 f   Kernel32.obj
 0001:0000154f       ??3@YAXPAXI@Z              1000254f f   MSVCRT:delete_scalar_size.obj
 0001:0000155d       ??_U@YAPAXI@Z              1000255d f   MSVCRT:new_array.obj
 0001:00001566       @__security_check_cookie@4 10002566 f   MSVCRT:secchk.obj
 0001:000018b4       __DllMainCRTStartup@12     100028b4 f   MSVCRT:dll_dllmain.obj
 0001:000018d7       ??3@YAXPAX@Z               100028d7 f   MSVCRT:delete_scalar.obj
 0001:000018dc       ??2@YAPAXI@Z               100028dc f   MSVCRT:new_scalar.obj
 0001:0000190c       ___raise_securityfailure   1000290c f   MSVCRT:gs_report.obj
 0001:00001934       ___report_gsfailure        10002934 f   MSVCRT:gs_report.obj
 0001:00001a7b       ___security_init_cookie    10002a7b f   MSVCRT:gs_support.obj
 0001:00001ac6       _DllMain@12                10002ac6 f   MSVCRT:dll_dllmain_stub.obj
 0001:00001ae8       ?__scrt_initialize_type_info@@YAXXZ 10002ae8 f   MSVCRT:tncleanup.obj
 0001:00001af4       ?__scrt_uninitialize_type_info@@YAXXZ 10002af4 f   MSVCRT:tncleanup.obj
 0001:00001b00       ___local_stdio_printf_options 10002b00 f i MSVCRT:default_local_stdio_options.obj
 0001:00001b06       ___local_stdio_scanf_options 10002b06 f i MSVCRT:default_local_stdio_options.obj
 0001:00001b0c       ___scrt_initialize_default_local_stdio_options 10002b0c f   MSVCRT:default_local_stdio_options.obj
 0001:00001b6d       ___scrt_acquire_startup_lock 10002b6d f   MSVCRT:utility.obj
 0001:00001b9f       ___scrt_dllmain_after_initialize_c 10002b9f f   MSVCRT:utility.obj
 0001:00001bca       ___scrt_dllmain_before_initialize_c 10002bca f   MSVCRT:utility.obj
 0001:00001bd8       ___scrt_dllmain_crt_thread_attach 10002bd8 f   MSVCRT:utility.obj
 0001:00001bf7       ___scrt_dllmain_crt_thread_detach 10002bf7 f   MSVCRT:utility.obj
 0001:00001c04       ___scrt_dllmain_exception_filter 10002c04 f   MSVCRT:utility.obj
 0001:00001c38       ___scrt_dllmain_uninitialize_c 10002c38 f   MSVCRT:utility.obj
 0001:00001c5b       ___scrt_dllmain_uninitialize_critical 10002c5b f   MSVCRT:utility.obj
 0001:00001c68       ___scrt_initialize_crt     10002c68 f   MSVCRT:utility.obj
 0001:00001ca1       ___scrt_initialize_onexit_tables 10002ca1 f   MSVCRT:utility.obj
 0001:00001d28       ___scrt_is_nonwritable_in_current_image 10002d28 f   MSVCRT:utility.obj
 0001:00001dbc       ___scrt_release_startup_lock 10002dbc f   MSVCRT:utility.obj
 0001:00001dd9       ___scrt_uninitialize_crt   10002dd9 f   MSVCRT:utility.obj
 0001:00001e01       ___scrt_get_dyn_tls_init_callback 10002e01 f   MSVCRT:dyn_tls_init.obj
 0001:00001e07       ___scrt_fastfail           10002e07 f   MSVCRT:utility_desktop.obj
 0001:00001f22       __crt_debugger_hook        10002f22 f   MSVCRT:utility_desktop.obj
 0001:00001f2a       __RTC_Initialize           10002f2a f   MSVCRT:initsect.obj
 0001:00001f56       __RTC_Terminate            10002f56 f   MSVCRT:initsect.obj
 0001:00001f90       __SEH_prolog4              10002f90 f   MSVCRT:sehprolg4.obj
 0001:00001fd5       __except_handler4          10002fd5 f   MSVCRT:chandler4gs.obj
 0001:00002004       @_guard_check_icall_nop@4  10003004 f i MSVCRT:guard_support.obj
 0001:00002007       ??0bad_alloc@std@@QAE@ABV01@@Z 10003007 f i MSVCRT:throw_bad_alloc.obj
 0001:00002022       ??0bad_alloc@std@@QAE@XZ   10003022 f i MSVCRT:throw_bad_alloc.obj
 0001:0000203a       ??0bad_array_new_length@std@@QAE@ABV01@@Z 1000303a f i MSVCRT:throw_bad_alloc.obj
 0001:00002055       ??0bad_array_new_length@std@@QAE@XZ 10003055 f i MSVCRT:throw_bad_alloc.obj
 0001:0000206d       ??0exception@std@@QAE@ABV01@@Z 1000306d f i MSVCRT:throw_bad_alloc.obj
 0001:00002099       ??1bad_alloc@std@@UAE@XZ   10003099 f i MSVCRT:throw_bad_alloc.obj
 0001:00002099       ??1bad_array_new_length@std@@UAE@XZ 10003099 f i MSVCRT:throw_bad_alloc.obj
 0001:000020aa       ??_Ebad_alloc@std@@UAEPAXI@Z 100030aa f i MSVCRT:throw_bad_alloc.obj
 0001:000020aa       ??_Ebad_array_new_length@std@@UAEPAXI@Z 100030aa f i MSVCRT:throw_bad_alloc.obj
 0001:000020aa       ??_Eexception@std@@UAEPAXI@Z 100030aa f i MSVCRT:throw_bad_alloc.obj
 0001:000020aa       ??_Gbad_alloc@std@@UAEPAXI@Z 100030aa f i MSVCRT:throw_bad_alloc.obj
 0001:000020aa       ??_Gbad_array_new_length@std@@UAEPAXI@Z 100030aa f i MSVCRT:throw_bad_alloc.obj
 0001:000020aa       ??_Gexception@std@@UAEPAXI@Z 100030aa f i MSVCRT:throw_bad_alloc.obj
 0001:000020d7       ?__scrt_throw_std_bad_alloc@@YAXXZ 100030d7 f   MSVCRT:throw_bad_alloc.obj
 0001:000020f4       ?__scrt_throw_std_bad_array_new_length@@YAXXZ 100030f4 f   MSVCRT:throw_bad_alloc.obj
 0001:00002111       ?what@exception@std@@UBEPBDXZ 10003111 f i MSVCRT:throw_bad_alloc.obj
 0001:0000211e       ___isa_available_init      1000311e f   MSVCRT:cpu_disp.obj
 0001:000022f2       __get_startup_argv_mode    100032f2 f   MSVCRT:argv_mode.obj
 0001:000022f6       ___scrt_is_ucrt_dll_in_use 100032f6 f   MSVCRT:ucrt_detection.obj
 0001:00002302       ??_Etype_info@@UAEPAXI@Z   10003302 f i MSVCRT:std_type_info_static.obj
 0001:00002302       ??_Gtype_info@@UAEPAXI@Z   10003302 f i MSVCRT:std_type_info_static.obj
 0001:00002325       ___std_type_info_destroy_list 10003325 f   vcruntime:VCRUNTIME140.dll
 0001:0000232b       _memset                    1000332b f   vcruntime:VCRUNTIME140.dll
 0001:00002331       __except_handler4_common   10003331 f   vcruntime:VCRUNTIME140.dll
 0001:00002337       ___std_exception_copy      10003337 f   vcruntime:VCRUNTIME140.dll
 0001:0000233d       ___std_exception_destroy   1000333d f   vcruntime:VCRUNTIME140.dll
 0001:00002343       __CxxThrowException@8      10003343 f   vcruntime:VCRUNTIME140.dll
 0001:00002349       __initterm                 10003349 f   ucrt:api-ms-win-crt-runtime-l1-1-0.dll
 0001:0000234f       __initterm_e               1000334f f   ucrt:api-ms-win-crt-runtime-l1-1-0.dll
 0001:00002355       _free                      10003355 f   ucrt:api-ms-win-crt-heap-l1-1-0.dll
 0001:0000235b       __callnewh                 1000335b f   ucrt:api-ms-win-crt-heap-l1-1-0.dll
 0001:00002361       _malloc                    10003361 f   ucrt:api-ms-win-crt-heap-l1-1-0.dll
 0001:00002367       __seh_filter_dll           10003367 f   ucrt:api-ms-win-crt-runtime-l1-1-0.dll
 0001:0000236d       __configure_narrow_argv    1000336d f   ucrt:api-ms-win-crt-runtime-l1-1-0.dll
 0001:00002373       __initialize_narrow_environment 10003373 f   ucrt:api-ms-win-crt-runtime-l1-1-0.dll
 0001:00002379       __initialize_onexit_table  10003379 f   ucrt:api-ms-win-crt-runtime-l1-1-0.dll
 0001:0000237f       __execute_onexit_table     1000337f f   ucrt:api-ms-win-crt-runtime-l1-1-0.dll
 0001:00002385       __cexit                    10003385 f   ucrt:api-ms-win-crt-runtime-l1-1-0.dll
 0001:0000238b       ___acrt_initialize         1000338b f   MSVCRT:ucrt_stubs.obj
 0001:0000238b       ___acrt_thread_attach      1000338b f   MSVCRT:ucrt_stubs.obj
 0001:0000238b       ___acrt_thread_detach      1000338b f   MSVCRT:ucrt_stubs.obj
 0001:0000238b       ___acrt_uninitialize       1000338b f   MSVCRT:ucrt_stubs.obj
 0001:0000238b       ___acrt_uninitialize_critical 1000338b f   MSVCRT:ucrt_stubs.obj
 0001:0000238b       ___scrt_stub_for_acrt_initialize 1000338b f   MSVCRT:ucrt_stubs.obj
 0001:0000238b       ___scrt_stub_for_acrt_thread_attach 1000338b f   MSVCRT:ucrt_stubs.obj
 0001:0000238b       ___scrt_stub_for_acrt_thread_detach 1000338b f   MSVCRT:ucrt_stubs.obj
 0001:0000238b       ___scrt_stub_for_acrt_uninitialize 1000338b f   MSVCRT:ucrt_stubs.obj
 0001:0000238b       ___scrt_stub_for_acrt_uninitialize_critical 1000338b f   MSVCRT:ucrt_stubs.obj
 0001:0000238b       ___vcrt_initialize         1000338b f   MSVCRT:ucrt_stubs.obj
 0001:0000238b       ___vcrt_thread_attach      1000338b f   MSVCRT:ucrt_stubs.obj
 0001:0000238b       ___vcrt_thread_detach      1000338b f   MSVCRT:ucrt_stubs.obj
 0001:0000238b       ___vcrt_uninitialize       1000338b f   MSVCRT:ucrt_stubs.obj
 0001:0000238b       ___vcrt_uninitialize_critical 1000338b f   MSVCRT:ucrt_stubs.obj
 0001:0000238e       ___scrt_stub_for_is_c_termination_complete 1000338e f   MSVCRT:ucrt_stubs.obj
 0001:0000238e       __is_c_termination_complete 1000338e f   MSVCRT:ucrt_stubs.obj
 0001:00002391       __filter_x86_sse2_floating_point_exception 10003391 f   MSVCRT:x86_exception_filter.obj
 0001:00002391       __filter_x86_sse2_floating_point_exception_default 10003391 f   MSVCRT:x86_exception_filter.obj
 0002:00000000       __imp__GetStdHandle@4      10004000     kernel32:KERNEL32.dll
 0002:00000004       __imp__GetLastError@0      10004004     kernel32:KERNEL32.dll
 0002:00000008       __imp__WaitForSingleObject@8 10004008     kernel32:KERNEL32.dll
 0002:0000000c       __imp__GetConsoleMode@8    1000400c     kernel32:KERNEL32.dll
 0002:00000010       __imp__SetConsoleMode@8    10004010     kernel32:KERNEL32.dll
 0002:00000014       __imp__ReadConsoleInputW@16 10004014     kernel32:KERNEL32.dll
 0002:00000018       __imp__WriteConsoleW@20    10004018     kernel32:KERNEL32.dll
 0002:0000001c       __imp__FillConsoleOutputCharacterA@20 1000401c     kernel32:KERNEL32.dll
 0002:00000020       __imp__FillConsoleOutputAttribute@20 10004020     kernel32:KERNEL32.dll
 0002:00000024       __imp__GetConsoleScreenBufferInfo@8 10004024     kernel32:KERNEL32.dll
 0002:00000028       __imp__SetConsoleCursorPosition@8 10004028     kernel32:KERNEL32.dll
 0002:0000002c       __imp__SetConsoleTextAttribute@8 1000402c     kernel32:KERNEL32.dll
 0002:00000030       __imp__ScrollConsoleScreenBufferA@20 10004030     kernel32:KERNEL32.dll
 0002:00000034       __imp__SetConsoleTitleA@4  10004034     kernel32:KERNEL32.dll
 0002:00000038       __imp__UnhandledExceptionFilter@4 10004038     kernel32:KERNEL32.dll
 0002:0000003c       __imp__SetUnhandledExceptionFilter@4 1000403c     kernel32:KERNEL32.dll
 0002:00000040       __imp__GetCurrentProcess@0 10004040     kernel32:KERNEL32.dll
 0002:00000044       __imp__TerminateProcess@8  10004044     kernel32:KERNEL32.dll
 0002:00000048       __imp__IsProcessorFeaturePresent@4 10004048     kernel32:KERNEL32.dll
 0002:0000004c       __imp__QueryPerformanceCounter@4 1000404c     kernel32:KERNEL32.dll
 0002:00000050       __imp__GetCurrentProcessId@0 10004050     kernel32:KERNEL32.dll
 0002:00000054       __imp__GetCurrentThreadId@0 10004054     kernel32:KERNEL32.dll
 0002:00000058       __imp__GetSystemTimeAsFileTime@4 10004058     kernel32:KERNEL32.dll
 0002:0000005c       __imp__DisableThreadLibraryCalls@4 1000405c     kernel32:KERNEL32.dll
 0002:00000060       __imp__InitializeSListHead@4 10004060     kernel32:KERNEL32.dll
 0002:00000064       __imp__IsDebuggerPresent@0 10004064     kernel32:KERNEL32.dll
 0002:00000068       \177KERNEL32_NULL_THUNK_DATA 10004068     kernel32:KERNEL32.dll
 0002:0000006c       __imp____std_type_info_destroy_list 1000406c     vcruntime:VCRUNTIME140.dll
 0002:00000070       __imp__memset              10004070     vcruntime:VCRUNTIME140.dll
 0002:00000074       __imp___except_handler4_common 10004074     vcruntime:VCRUNTIME140.dll
 0002:00000078       __imp____std_exception_copy 10004078     vcruntime:VCRUNTIME140.dll
 0002:0000007c       __imp____std_exception_destroy 1000407c     vcruntime:VCRUNTIME140.dll
 0002:00000080       __imp___CxxThrowException@8 10004080     vcruntime:VCRUNTIME140.dll
 0002:00000084       \177VCRUNTIME140_NULL_THUNK_DATA 10004084     vcruntime:VCRUNTIME140.dll
 0002:00000088       __imp__malloc              10004088     ucrt:api-ms-win-crt-heap-l1-1-0.dll
 0002:0000008c       __imp___callnewh           1000408c     ucrt:api-ms-win-crt-heap-l1-1-0.dll
 0002:00000090       __imp__free                10004090     ucrt:api-ms-win-crt-heap-l1-1-0.dll
 0002:00000094       \177api-ms-win-crt-heap-l1-1-0_NULL_THUNK_DATA 10004094     ucrt:api-ms-win-crt-heap-l1-1-0.dll
 0002:00000098       __imp___initterm           10004098     ucrt:api-ms-win-crt-runtime-l1-1-0.dll
 0002:0000009c       __imp___seh_filter_dll     1000409c     ucrt:api-ms-win-crt-runtime-l1-1-0.dll
 0002:000000a0       __imp___configure_narrow_argv 100040a0     ucrt:api-ms-win-crt-runtime-l1-1-0.dll
 0002:000000a4       __imp___initialize_narrow_environment 100040a4     ucrt:api-ms-win-crt-runtime-l1-1-0.dll
 0002:000000a8       __imp___initialize_onexit_table 100040a8     ucrt:api-ms-win-crt-runtime-l1-1-0.dll
 0002:000000ac       __imp___execute_onexit_table 100040ac     ucrt:api-ms-win-crt-runtime-l1-1-0.dll
 0002:000000b0       __imp___cexit              100040b0     ucrt:api-ms-win-crt-runtime-l1-1-0.dll
 0002:000000b4       __imp___initterm_e         100040b4     ucrt:api-ms-win-crt-runtime-l1-1-0.dll
 0002:000000b8       \177api-ms-win-crt-runtime-l1-1-0_NULL_THUNK_DATA 100040b8     ucrt:api-ms-win-crt-runtime-l1-1-0.dll
 0002:000000bc       ___guard_check_icall_fptr  100040bc     MSVCRT:guard_support.obj
 0002:000000c0       ___castguard_check_failure_os_handled_fptr 100040c0     MSVCRT:guard_support.obj
 0002:000000c4       ___xc_a                    100040c4     MSVCRT:initializers.obj
 0002:000000c8       ___xc_z                    100040c8     MSVCRT:initializers.obj
 0002:000000cc       ___xi_a                    100040cc     MSVCRT:initializers.obj
 0002:000000d0       ___xi_z                    100040d0     MSVCRT:initializers.obj
 0002:000000d4       ___xp_a                    100040d4     MSVCRT:initializers.obj
 0002:000000d8       ___xp_z                    100040d8     MSVCRT:initializers.obj
 0002:000000dc       ___xt_a                    100040dc     MSVCRT:initializers.obj
 0002:000000e0       ___xt_z                    100040e0     MSVCRT:initializers.obj
 0002:000000e8       ??_C@_0DF@LIHHLEHB@jdk?1internal?1org?1jline?1terminal@ 100040e8     Kernel32.obj
 0002:00000120       ??_C@_04OHLIFDMD@?$CIJ?$CJV@ 10004120     Kernel32.obj
 0002:00000128       ??_C@_06FALKBLGB@?$DMinit?$DO@ 10004128     Kernel32.obj
 0002:00000130       ??_C@_01LELAEKIP@J@        10004130     Kernel32.obj
 0002:00000134       ??_C@_05MFEJDJP@value@     10004134     Kernel32.obj
 0002:00000140       ??_C@_0EA@DDCNJKJC@jdk?1internal?1org?1jline?1terminal@ 10004140     Kernel32.obj
 0002:00000180       ??_C@_0DM@MBLFOGAB@jdk?1internal?1org?1jline?1terminal@ 10004180     Kernel32.obj
 0002:000001bc       ??_C@_01JPJNBJEM@I@        100041bc     Kernel32.obj
 0002:000001c0       ??_C@_0EA@EMLEKAEK@jdk?1internal?1org?1jline?1terminal@ 100041c0     Kernel32.obj
 0002:00000200       ??_C@_03GAEACAIP@?$CI?$CJV@ 10004200     Kernel32.obj
 0002:00000208       ??_C@_0EC@GLHGKIHD@Ljdk?1internal?1org?1jline?1termina@ 10004208     Kernel32.obj
 0002:0000024c       ??_C@_05KAAPIFDI@uChar@    1000424c     Kernel32.obj
 0002:00000254       ??_C@_01CPLAODJH@S@        10004254     Kernel32.obj
 0002:00000258       ??_C@_0L@PLFFHFAH@Attributes@ 10004258     Kernel32.obj
 0002:00000268       ??_C@_0EK@EAOKBDCN@jdk?1internal?1org?1jline?1terminal@ 10004268     Kernel32.obj
 0002:000002b4       ??_C@_06HDDMAKPI@dwSize@   100042b4     Kernel32.obj
 0002:000002bc       ??_C@_01POHCFINO@Z@        100042bc     Kernel32.obj
 0002:000002c0       ??_C@_08DHPIEJHJ@bVisible@ 100042c0     Kernel32.obj
 0002:000002d0       ??_C@_0FB@CKOMJLPB@jdk?1internal?1org?1jline?1terminal@ 100042d0     Kernel32.obj
 0002:00000324       ??_C@_0DO@KLOLFBPB@Ljdk?1internal?1org?1jline?1termina@ 10004324     Kernel32.obj
 0002:00000364       ??_C@_0BB@GCKPAHKE@dwCursorPosition@ 10004364     Kernel32.obj
 0002:00000378       ??_C@_0M@LLNFGKPP@wAttributes@ 10004378     Kernel32.obj
 0002:00000388       ??_C@_0ED@GDPBCFCF@Ljdk?1internal?1org?1jline?1termina@ 10004388     Kernel32.obj
 0002:000003cc       ??_C@_08EGJHMBFD@srWindow@ 100043cc     Kernel32.obj
 0002:000003d8       ??_C@_0BE@DLBDILN@dwMaximumWindowSize@ 100043d8     Kernel32.obj
 0002:000003ec       ??_C@_0DM@IOLEMLOB@jdk?1internal?1org?1jline?1terminal@ 100043ec     Kernel32.obj
 0002:00000428       ??_C@_01MMEEDKFM@X@        10004428     Kernel32.obj
 0002:0000042c       ??_C@_01NFFPALBN@Y@        1000442c     Kernel32.obj
 0002:00000430       ??_C@_0ED@KEABPHEC@jdk?1internal?1org?1jline?1terminal@ 10004430     Kernel32.obj
 0002:00000474       ??_C@_09KDLBEGCN@EventType@ 10004474     Kernel32.obj
 0002:00000480       ??_C@_0FA@EPHOAIKB@Ljdk?1internal?1org?1jline?1termina@ 10004480     Kernel32.obj
 0002:000004d0       ??_C@_05GCNIINAF@Event@    100044d0     Kernel32.obj
 0002:000004d8       ??_C@_0EO@ENJPMKIB@jdk?1internal?1org?1jline?1terminal@ 100044d8     Kernel32.obj
 0002:00000528       ??_C@_0EJ@KAFKPAON@Ljdk?1internal?1org?1jline?1termina@ 10004528     Kernel32.obj
 0002:00000574       ??_C@_08IICPJOPF@KeyEvent@ 10004574     Kernel32.obj
 0002:00000580       ??_C@_0EL@NEMNNEIM@Ljdk?1internal?1org?1jline?1termina@ 10004580     Kernel32.obj
 0002:000005cc       ??_C@_0L@MEMIOFPE@MouseEvent@ 100045cc     Kernel32.obj
 0002:000005d8       ??_C@_0FC@GJCMFPEB@Ljdk?1internal?1org?1jline?1termina@ 100045d8     Kernel32.obj
 0002:0000062c       ??_C@_0BG@FDJGLIMD@WindowBufferSizeEvent@ 1000462c     Kernel32.obj
 0002:00000648       ??_C@_0EK@GINBNDHB@Ljdk?1internal?1org?1jline?1termina@ 10004648     Kernel32.obj
 0002:00000694       ??_C@_09DGBBEBCO@MenuEvent@ 10004694     Kernel32.obj
 0002:000006a0       ??_C@_0EL@NEOCEPBL@Ljdk?1internal?1org?1jline?1termina@ 100046a0     Kernel32.obj
 0002:000006ec       ??_C@_0L@PKFCPJDI@FocusEvent@ 100046ec     Kernel32.obj
 0002:000006f8       ??_C@_0EH@LAMOGNLH@jdk?1internal?1org?1jline?1terminal@ 100046f8     Kernel32.obj
 0002:00000740       ??_C@_08IOMBICKD@bKeyDown@ 10004740     Kernel32.obj
 0002:0000074c       ??_C@_0N@OFEBLKAO@wRepeatCount@ 1000474c     Kernel32.obj
 0002:0000075c       ??_C@_0BA@ODMGPHEG@wVirtualKeyCode@ 1000475c     Kernel32.obj
 0002:0000076c       ??_C@_0BB@GLFALPCM@wVirtualScanCode@ 1000476c     Kernel32.obj
 0002:00000780       ??_C@_0BC@CPLAFJNJ@dwControlKeyState@ 10004780     Kernel32.obj
 0002:00000798       ??_C@_0EJ@KJENNMFH@jdk?1internal?1org?1jline?1terminal@ 10004798     Kernel32.obj
 0002:000007e4       ??_C@_0BA@CLCFHGAI@dwMousePosition@ 100047e4     Kernel32.obj
 0002:000007f4       ??_C@_0O@OBJAOKMC@dwButtonState@ 100047f4     Kernel32.obj
 0002:00000804       ??_C@_0N@LGDKLHCN@dwEventFlags@ 10004804     Kernel32.obj
 0002:00000818       ??_C@_0FA@ELBPHOIL@jdk?1internal?1org?1jline?1terminal@ 10004818     Kernel32.obj
 0002:00000868       ??_C@_0EI@HEDGJHGB@jdk?1internal?1org?1jline?1terminal@ 10004868     Kernel32.obj
 0002:000008b0       ??_C@_0M@ILCOGF@dwCommandId@ 100048b0     Kernel32.obj
 0002:000008c0       ??_C@_0EJ@IGNGELFH@jdk?1internal?1org?1jline?1terminal@ 100048c0     Kernel32.obj
 0002:0000090c       ??_C@_09LPEMLFBO@bSetFocus@ 1000490c     Kernel32.obj
 0002:00000918       ??_C@_0EB@FEHKODDE@jdk?1internal?1org?1jline?1terminal@ 10004918     Kernel32.obj
 0002:0000095c       ??_C@_04KPCPLBPL@Left@     1000495c     Kernel32.obj
 0002:00000964       ??_C@_03PGGAENPN@Top@      10004964     Kernel32.obj
 0002:00000968       ??_C@_05DADPALEM@Right@    10004968     Kernel32.obj
 0002:00000970       ??_C@_06DDHCBBGN@Bottom@   10004970     Kernel32.obj
 0002:00000978       ??_C@_0EA@CDONDDCN@jdk?1internal?1org?1jline?1terminal@ 10004978     Kernel32.obj
 0002:000009b8       ??_C@_01GFHCPBMG@C@        100049b8     Kernel32.obj
 0002:000009bc       ??_C@_0M@PBJKDIHH@UnicodeChar@ 100049bc     Kernel32.obj
 0002:000009c8       __pDefaultRawDllMain       100049c8     MSVCRT:dll_dllmain.obj
 0002:000009c8       __pRawDllMain              100049c8     MSVCRT:dll_dllmain.obj
 0002:000009d8       ??_7exception@std@@6B@     100049d8     MSVCRT:throw_bad_alloc.obj
 0002:000009e0       ??_C@_0BC@EOODALEL@Unknown?5exception@ 100049e0     MSVCRT:throw_bad_alloc.obj
 0002:000009f8       ??_7bad_alloc@std@@6B@     100049f8     MSVCRT:throw_bad_alloc.obj
 0002:00000a00       ??_C@_0P@GHFPNOJB@bad?5allocation@ 10004a00     MSVCRT:throw_bad_alloc.obj
 0002:00000a14       ??_7bad_array_new_length@std@@6B@ 10004a14     MSVCRT:throw_bad_alloc.obj
 0002:00000a1c       ??_C@_0BF@KINCDENJ@bad?5array?5new?5length@ 10004a1c     MSVCRT:throw_bad_alloc.obj
 0002:00000a38       ??_7type_info@@6B@         10004a38     MSVCRT:std_type_info_static.obj
 0002:00000a40       __load_config_used         10004a40     MSVCRT:loadcfg.obj
 0002:00000b80       ??_R4exception@std@@6B@    10004b80     MSVCRT:throw_bad_alloc.obj
 0002:00000b94       ??_R3exception@std@@8      10004b94     MSVCRT:throw_bad_alloc.obj
 0002:00000ba4       ??_R2exception@std@@8      10004ba4     MSVCRT:throw_bad_alloc.obj
 0002:00000bac       ??_R1A@?0A@EA@exception@std@@8 10004bac     MSVCRT:throw_bad_alloc.obj
 0002:00000bc8       ??_R4bad_alloc@std@@6B@    10004bc8     MSVCRT:throw_bad_alloc.obj
 0002:00000bdc       ??_R3bad_alloc@std@@8      10004bdc     MSVCRT:throw_bad_alloc.obj
 0002:00000bec       ??_R2bad_alloc@std@@8      10004bec     MSVCRT:throw_bad_alloc.obj
 0002:00000bf8       ??_R1A@?0A@EA@bad_alloc@std@@8 10004bf8     MSVCRT:throw_bad_alloc.obj
 0002:00000c14       ??_R4bad_array_new_length@std@@6B@ 10004c14     MSVCRT:throw_bad_alloc.obj
 0002:00000c28       ??_R3bad_array_new_length@std@@8 10004c28     MSVCRT:throw_bad_alloc.obj
 0002:00000c38       ??_R2bad_array_new_length@std@@8 10004c38     MSVCRT:throw_bad_alloc.obj
 0002:00000c48       ??_R1A@?0A@EA@bad_array_new_length@std@@8 10004c48     MSVCRT:throw_bad_alloc.obj
 0002:00000c64       ??_R4type_info@@6B@        10004c64     MSVCRT:std_type_info_static.obj
 0002:00000c78       ??_R3type_info@@8          10004c78     MSVCRT:std_type_info_static.obj
 0002:00000c88       ??_R2type_info@@8          10004c88     MSVCRT:std_type_info_static.obj
 0002:00000c90       ??_R1A@?0A@EA@type_info@@8 10004c90     MSVCRT:std_type_info_static.obj
 0002:00000cac       ___safe_se_handler_table   10004cac     <linker-defined>
 0002:00000cb0       ___volatile_metadata       10004cb0     <linker-defined>
 0002:00000fdc       ___rtc_iaa                 10004fdc     MSVCRT:initsect.obj
 0002:00000fe0       ___rtc_izz                 10004fe0     MSVCRT:initsect.obj
 0002:00000fe4       ___rtc_taa                 10004fe4     MSVCRT:initsect.obj
 0002:00000fe8       ___rtc_tzz                 10004fe8     MSVCRT:initsect.obj
 0002:00001074       __TI2?AVbad_alloc@std@@    10005074     MSVCRT:throw_bad_alloc.obj
 0002:00001084       __CTA2?AVbad_alloc@std@@   10005084     MSVCRT:throw_bad_alloc.obj
 0002:00001090       __CT??_R0?AVbad_alloc@std@@@8??0bad_alloc@std@@QAE@ABV01@@Z12 10005090     MSVCRT:throw_bad_alloc.obj
 0002:000010ac       __CT??_R0?AVexception@std@@@8??0exception@std@@QAE@ABV01@@Z12 100050ac     MSVCRT:throw_bad_alloc.obj
 0002:000010c8       __TI3?AVbad_array_new_length@std@@ 100050c8     MSVCRT:throw_bad_alloc.obj
 0002:000010d8       __CTA3?AVbad_array_new_length@std@@ 100050d8     MSVCRT:throw_bad_alloc.obj
 0002:000010e8       __CT??_R0?AVbad_array_new_length@std@@@8??0bad_array_new_length@std@@QAE@ABV01@@Z12 100050e8     MSVCRT:throw_bad_alloc.obj
 0002:00001688       __IMPORT_DESCRIPTOR_KERNEL32 10005688     kernel32:KERNEL32.dll
 0002:0000169c       __IMPORT_DESCRIPTOR_VCRUNTIME140 1000569c     vcruntime:VCRUNTIME140.dll
 0002:000016b0       __IMPORT_DESCRIPTOR_api-ms-win-crt-runtime-l1-1-0 100056b0     ucrt:api-ms-win-crt-runtime-l1-1-0.dll
 0002:000016c4       __IMPORT_DESCRIPTOR_api-ms-win-crt-heap-l1-1-0 100056c4     ucrt:api-ms-win-crt-heap-l1-1-0.dll
 0002:000016d8       __NULL_IMPORT_DESCRIPTOR   100056d8     kernel32:KERNEL32.dll
 0003:00000000       ___security_cookie_complement 10006000     MSVCRT:gs_cookie.obj
 0003:00000004       ___security_cookie         10006004     MSVCRT:gs_cookie.obj
 0003:00000008       ___scrt_native_dllmain_reason 10006008     MSVCRT:utility.obj
 0003:00000010       ___isa_enabled             10006010     MSVCRT:cpu_disp.obj
 0003:00000014       ___scrt_ucrt_dll_is_in_use 10006014     MSVCRT:ucrt_stubs.obj
 0003:00000018       ??_R0?AVbad_alloc@std@@@8  10006018     MSVCRT:throw_bad_alloc.obj
 0003:00000034       ??_R0?AVexception@std@@@8  10006034     MSVCRT:throw_bad_alloc.obj
 0003:00000050       ??_R0?AVbad_array_new_length@std@@@8 10006050     MSVCRT:throw_bad_alloc.obj
 0003:00000078       ??_R0?AVtype_info@@@8      10006078     MSVCRT:std_type_info_static.obj
 0003:000004c8       ?__type_info_root_node@@3U__type_info_node@@A 100064c8     MSVCRT:tncleanup.obj
 0003:000004d0       ?_OptionsStorage@?1??__local_stdio_printf_options@@9@4_KA 100064d0     MSVCRT:default_local_stdio_options.obj
 0003:000004d8       ?_OptionsStorage@?1??__local_stdio_scanf_options@@9@4_KA 100064d8     MSVCRT:default_local_stdio_options.obj
 0003:000004e0       ___scrt_current_native_startup_state 100064e0     MSVCRT:utility.obj
 0003:000004e4       ___scrt_native_startup_lock 100064e4     MSVCRT:utility.obj
 0003:00000504       ___scrt_debugger_hook_flag 10006504     MSVCRT:utility_desktop.obj
 0003:00000508       ___isa_available           10006508     MSVCRT:cpu_disp.obj
 0003:0000050c       ___favor                   1000650c     MSVCRT:cpu_disp.obj
 0003:00000510       ___dyn_tls_init_callback   10006510     <common>

 entry point at        0001:000018b4

 Static symbols

 0000:ffff7000       .debug$S                   10000000     le.exp
 0000:ffff7000       .debug$S                   10000000     vcruntime:VCRUNTIME140.dll
 0000:ffff7000       .debug$S                   10000000     vcruntime:VCRUNTIME140.dll
 0000:ffff7000       .debug$S                   10000000     vcruntime:VCRUNTIME140.dll
 0000:ffff7000       .debug$S                   10000000     vcruntime:VCRUNTIME140.dll
 0000:ffff7000       .debug$S                   10000000     vcruntime:VCRUNTIME140.dll
 0000:ffff7000       .debug$S                   10000000     vcruntime:VCRUNTIME140.dll
 0000:ffff7000       .debug$S                   10000000     vcruntime:VCRUNTIME140.dll
 0000:ffff7000       .debug$S                   10000000     vcruntime:VCRUNTIME140.dll
 0000:ffff7000       .debug$S                   10000000     ucrt:api-ms-win-crt-heap-l1-1-0.dll
 0000:ffff7000       .debug$S                   10000000     ucrt:api-ms-win-crt-heap-l1-1-0.dll
 0000:ffff7000       .debug$S                   10000000     ucrt:api-ms-win-crt-heap-l1-1-0.dll
 0000:ffff7000       .debug$S                   10000000     ucrt:api-ms-win-crt-runtime-l1-1-0.dll
 0000:ffff7000       .debug$S                   10000000     ucrt:api-ms-win-crt-runtime-l1-1-0.dll
 0000:ffff7000       .debug$S                   10000000     ucrt:api-ms-win-crt-runtime-l1-1-0.dll
 0000:ffff7000       .debug$S                   10000000     ucrt:api-ms-win-crt-runtime-l1-1-0.dll
 0000:ffff7000       .debug$S                   10000000     ucrt:api-ms-win-crt-runtime-l1-1-0.dll
 0000:ffff7000       .debug$S                   10000000     ucrt:api-ms-win-crt-runtime-l1-1-0.dll
 0000:ffff7000       .debug$S                   10000000     ucrt:api-ms-win-crt-runtime-l1-1-0.dll
 0000:ffff7000       .debug$S                   10000000     ucrt:api-ms-win-crt-runtime-l1-1-0.dll
 0000:ffff7000       .debug$S                   10000000     ucrt:api-ms-win-crt-runtime-l1-1-0.dll
 0000:ffff7000       .debug$S                   10000000     ucrt:api-ms-win-crt-runtime-l1-1-0.dll
 0000:ffff7000       .debug$S                   10000000     ucrt:api-ms-win-crt-runtime-l1-1-0.dll
 0000:ffff7000       .debug$S                   10000000     ucrt:api-ms-win-crt-runtime-l1-1-0.dll
 0000:ffff7000       .debug$S                   10000000     kernel32:KERNEL32.dll
 0000:ffff7000       .debug$S                   10000000     kernel32:KERNEL32.dll
 0000:ffff7000       .debug$S                   10000000     kernel32:KERNEL32.dll
 0000:ffff7000       .debug$S                   10000000     kernel32:KERNEL32.dll
 0000:ffff7000       .debug$S                   10000000     kernel32:KERNEL32.dll
 0000:ffff7000       .debug$S                   10000000     kernel32:KERNEL32.dll
 0000:ffff7000       .debug$S                   10000000     kernel32:KERNEL32.dll
 0000:ffff7000       .debug$S                   10000000     kernel32:KERNEL32.dll
 0000:ffff7000       .debug$S                   10000000     kernel32:KERNEL32.dll
 0000:ffff7000       .debug$S                   10000000     kernel32:KERNEL32.dll
 0000:ffff7000       .debug$S                   10000000     kernel32:KERNEL32.dll
 0000:ffff7000       .debug$S                   10000000     kernel32:KERNEL32.dll
 0000:ffff7000       .debug$S                   10000000     kernel32:KERNEL32.dll
 0000:ffff7000       .debug$S                   10000000     kernel32:KERNEL32.dll
 0000:ffff7000       .debug$S                   10000000     kernel32:KERNEL32.dll
 0000:ffff7000       .debug$S                   10000000     kernel32:KERNEL32.dll
 0000:ffff7000       .debug$S                   10000000     kernel32:KERNEL32.dll
 0000:ffff7000       .debug$S                   10000000     kernel32:KERNEL32.dll
 0000:ffff7000       .debug$S                   10000000     kernel32:KERNEL32.dll
 0000:ffff7000       .debug$S                   10000000     kernel32:KERNEL32.dll
 0000:ffff7000       .debug$S                   10000000     kernel32:KERNEL32.dll
 0000:ffff7000       .debug$S                   10000000     kernel32:KERNEL32.dll
 0000:ffff7000       .debug$S                   10000000     kernel32:KERNEL32.dll
 0000:ffff7000       .debug$S                   10000000     kernel32:KERNEL32.dll
 0000:ffff7000       .debug$S                   10000000     kernel32:KERNEL32.dll
 0000:ffff7000       .debug$S                   10000000     kernel32:KERNEL32.dll
 0000:ffff7000       .debug$S                   10000000     kernel32:KERNEL32.dll
 0000:ffff7000       .debug$S                   10000000     kernel32:KERNEL32.dll
 0001:00001574       ?dllmain_crt_dispatch@@YGHQAUHINSTANCE__@@KQAX@Z 10002574 f   MSVCRT:dll_dllmain.obj
 0001:000015c7       ?dllmain_crt_process_attach@@YAHQAUHINSTANCE__@@QAX@Z 100025c7 f   MSVCRT:dll_dllmain.obj
 0001:000016ce       ?dllmain_crt_process_detach@@YAH_N@Z 100026ce f   MSVCRT:dll_dllmain.obj
 0001:0000177e       ?dllmain_dispatch@@YAHQAUHINSTANCE__@@KQAX@Z 1000277e f   MSVCRT:dll_dllmain.obj
 0001:00001889       ?dllmain_raw@@YGHQAUHINSTANCE__@@KQAX@Z 10002889 f   MSVCRT:dll_dllmain.obj
 0001:00001a2e       ___get_entropy             10002a2e f   MSVCRT:gs_support.obj
 0001:00001b29       ?find_pe_section@@YAPAU_IMAGE_SECTION_HEADER@@QAEI@Z 10002b29 f   MSVCRT:utility.obj
 0001:00001f90       $$000000                   10002f90     MSVCRT:sehprolg4.obj
 0002:000009cc       _GS_ExceptionPointers      100049cc     MSVCRT:gs_report.obj
 0002:00000ff0       __sehtable$?dllmain_crt_process_attach@@YAHQAUHINSTANCE__@@QAX@Z 10004ff0     MSVCRT:dll_dllmain.obj
 0002:00001010       __sehtable$?dllmain_crt_process_detach@@YAH_N@Z 10005010     MSVCRT:dll_dllmain.obj
 0002:00001038       __sehtable$?dllmain_dispatch@@YAHQAUHINSTANCE__@@KQAX@Z 10005038     MSVCRT:dll_dllmain.obj
 0002:00001058       __sehtable$___scrt_is_nonwritable_in_current_image 10005058     MSVCRT:utility.obj
 0002:00001110       .edata                     10005110     le.exp
 0002:00001138       rgpv                       10005138     le.exp
 0002:00001170       rgszName                   10005170     le.exp
 0002:000011a8       rgwOrd                     100051a8     le.exp
 0002:000011c4       szName                     100051c4     le.exp
 0002:000011cb       $N00001                    100051cb     le.exp
 0002:00001229       $N00002                    10005229     le.exp
 0002:00001287       $N00003                    10005287     le.exp
 0002:000012d9       $N00004                    100052d9     le.exp
 0002:00001337       $N00005                    10005337     le.exp
 0002:00001387       $N00006                    10005387     le.exp
 0002:000013db       $N00007                    100053db     le.exp
 0002:00001438       $N00008                    10005438     le.exp
 0002:00001494       $N00009                    10005494     le.exp
 0002:000014e6       $N00010                    100054e6     le.exp
 0002:00001541       $N00011                    10005541     le.exp
 0002:00001594       $N00012                    10005594     le.exp
 0002:000015eb       $N00013                    100055eb     le.exp
 0002:0000163c       $N00014                    1000563c     le.exp
 0002:00001a0c       .idata$6                   10005a0c     kernel32:KERNEL32.dll
 0002:00001aa6       .idata$6                   10005aa6     vcruntime:VCRUNTIME140.dll
 0002:00001b7c       .idata$6                   10005b7c     ucrt:api-ms-win-crt-runtime-l1-1-0.dll
 0002:00001b9e       .idata$6                   10005b9e     ucrt:api-ms-win-crt-heap-l1-1-0.dll
 0003:00000090       ?pointerClass@@3PAV_jclass@@A 10006090     Kernel32.obj
 0003:00000094       ?pointerConstructor@@3PAU_jmethodID@@A 10006094     Kernel32.obj
 0003:00000098       ?pointerValue@@3PAU_jfieldID@@A 10006098     Kernel32.obj
 0003:0000009c       ?intByReferenceClass@@3PAV_jclass@@A 1000609c     Kernel32.obj
 0003:000000a0       ?intByReferenceValue@@3PAU_jfieldID@@A 100060a0     Kernel32.obj
 0003:000000a4       ?lastErrorExceptionClass@@3PAV_jclass@@A 100060a4     Kernel32.obj
 0003:000000a8       ?lastErrorExceptionConstructor@@3PAU_jmethodID@@A 100060a8     Kernel32.obj
 0003:000000ac       ?CHAR_INFO_Class@@3PAV_jclass@@A 100060ac     Kernel32.obj
 0003:000000b0       ?CHAR_INFO_Constructor@@3PAU_jmethodID@@A 100060b0     Kernel32.obj
 0003:000000b4       ?CHAR_INFO_uChar@@3PAU_jfieldID@@A 100060b4     Kernel32.obj
 0003:000000b8       ?CHAR_INFO_Attributes@@3PAU_jfieldID@@A 100060b8     Kernel32.obj
 0003:000000bc       ?CONSOLE_CURSOR_INFO_Class@@3PAV_jclass@@A 100060bc     Kernel32.obj
 0003:000000c0       ?CONSOLE_CURSOR_INFO_Constructor@@3PAU_jmethodID@@A 100060c0     Kernel32.obj
 0003:000000c4       ?CONSOLE_CURSOR_INFO_dwSize@@3PAU_jfieldID@@A 100060c4     Kernel32.obj
 0003:000000c8       ?CONSOLE_CURSOR_INFO_bVisible@@3PAU_jfieldID@@A 100060c8     Kernel32.obj
 0003:000000cc       ?CONSOLE_SCREEN_BUFFER_INFO_Class@@3PAV_jclass@@A 100060cc     Kernel32.obj
 0003:000000d0       ?CONSOLE_SCREEN_BUFFER_INFO_Constructor@@3PAU_jmethodID@@A 100060d0     Kernel32.obj
 0003:000000d4       ?CONSOLE_SCREEN_BUFFER_INFO_dwSize@@3PAU_jfieldID@@A 100060d4     Kernel32.obj
 0003:000000d8       ?CONSOLE_SCREEN_BUFFER_INFO_dwCursorPosition@@3PAU_jfieldID@@A 100060d8     Kernel32.obj
 0003:000000dc       ?CONSOLE_SCREEN_BUFFER_INFO_wAttributes@@3PAU_jfieldID@@A 100060dc     Kernel32.obj
 0003:000000e0       ?CONSOLE_SCREEN_BUFFER_INFO_srWindow@@3PAU_jfieldID@@A 100060e0     Kernel32.obj
 0003:000000e4       ?CONSOLE_SCREEN_BUFFER_INFO_dwMaximumWindowSize@@3PAU_jfieldID@@A 100060e4     Kernel32.obj
 0003:000000e8       ?COORD_Class@@3PAV_jclass@@A 100060e8     Kernel32.obj
 0003:000000ec       ?COORD_Constructor@@3PAU_jmethodID@@A 100060ec     Kernel32.obj
 0003:000000f0       ?COORD_X@@3PAU_jfieldID@@A 100060f0     Kernel32.obj
 0003:000000f4       ?COORD_Y@@3PAU_jfieldID@@A 100060f4     Kernel32.obj
 0003:000000f8       ?INPUT_RECORD_Class@@3PAV_jclass@@A 100060f8     Kernel32.obj
 0003:000000fc       ?INPUT_RECORD_Constructor@@3PAU_jmethodID@@A 100060fc     Kernel32.obj
 0003:00000100       ?INPUT_RECORD_EventType@@3PAU_jfieldID@@A 10006100     Kernel32.obj
 0003:00000104       ?INPUT_RECORD_Event@@3PAU_jfieldID@@A 10006104     Kernel32.obj
 0003:00000108       ?EventUnion_Class@@3PAV_jclass@@A 10006108     Kernel32.obj
 0003:0000010c       ?EventUnion_Constructor@@3PAU_jmethodID@@A 1000610c     Kernel32.obj
 0003:00000110       ?EventUnion_KeyEvent@@3PAU_jfieldID@@A 10006110     Kernel32.obj
 0003:00000114       ?EventUnion_MouseEvent@@3PAU_jfieldID@@A 10006114     Kernel32.obj
 0003:00000118       ?EventUnion_WindowBufferSizeEvent@@3PAU_jfieldID@@A 10006118     Kernel32.obj
 0003:0000011c       ?EventUnion_MenuEvent@@3PAU_jfieldID@@A 1000611c     Kernel32.obj
 0003:00000120       ?EventUnion_FocusEvent@@3PAU_jfieldID@@A 10006120     Kernel32.obj
 0003:00000124       ?KEY_EVENT_RECORD_Class@@3PAV_jclass@@A 10006124     Kernel32.obj
 0003:00000128       ?KEY_EVENT_RECORD_Constructor@@3PAU_jmethodID@@A 10006128     Kernel32.obj
 0003:0000012c       ?KEY_EVENT_RECORD_bKeyDown@@3PAU_jfieldID@@A 1000612c     Kernel32.obj
 0003:00000130       ?KEY_EVENT_RECORD_wRepeatCount@@3PAU_jfieldID@@A 10006130     Kernel32.obj
 0003:00000134       ?KEY_EVENT_RECORD_wVirtualKeyCode@@3PAU_jfieldID@@A 10006134     Kernel32.obj
 0003:00000138       ?KEY_EVENT_RECORD_wVirtualScanCode@@3PAU_jfieldID@@A 10006138     Kernel32.obj
 0003:0000013c       ?KEY_EVENT_RECORD_uChar@@3PAU_jfieldID@@A 1000613c     Kernel32.obj
 0003:00000140       ?KEY_EVENT_RECORD_dwControlKeyState@@3PAU_jfieldID@@A 10006140     Kernel32.obj
 0003:00000144       ?MOUSE_EVENT_RECORD_Class@@3PAV_jclass@@A 10006144     Kernel32.obj
 0003:00000148       ?MOUSE_EVENT_RECORD_Constructor@@3PAU_jmethodID@@A 10006148     Kernel32.obj
 0003:0000014c       ?MOUSE_EVENT_RECORD_dwMousePosition@@3PAU_jfieldID@@A 1000614c     Kernel32.obj
 0003:00000150       ?MOUSE_EVENT_RECORD_dwButtonState@@3PAU_jfieldID@@A 10006150     Kernel32.obj
 0003:00000154       ?MOUSE_EVENT_RECORD_dwControlKeyState@@3PAU_jfieldID@@A 10006154     Kernel32.obj
 0003:00000158       ?MOUSE_EVENT_RECORD_dwEventFlags@@3PAU_jfieldID@@A 10006158     Kernel32.obj
 0003:0000015c       ?WINDOW_BUFFER_SIZE_RECORD_Class@@3PAV_jclass@@A 1000615c     Kernel32.obj
 0003:00000160       ?WINDOW_BUFFER_SIZE_RECORD_Constructor@@3PAU_jmethodID@@A 10006160     Kernel32.obj
 0003:00000164       ?WINDOW_BUFFER_SIZE_RECORD_dwSize@@3PAU_jfieldID@@A 10006164     Kernel32.obj
 0003:00000168       ?MENU_EVENT_RECORD_Class@@3PAV_jclass@@A 10006168     Kernel32.obj
 0003:0000016c       ?MENU_EVENT_RECORD_Constructor@@3PAU_jmethodID@@A 1000616c     Kernel32.obj
 0003:00000170       ?MENU_EVENT_RECORD_dwCommandId@@3PAU_jfieldID@@A 10006170     Kernel32.obj
 0003:00000174       ?FOCUS_EVENT_RECORD_Class@@3PAV_jclass@@A 10006174     Kernel32.obj
 0003:00000178       ?FOCUS_EVENT_RECORD_Constructor@@3PAU_jmethodID@@A 10006178     Kernel32.obj
 0003:0000017c       ?FOCUS_EVENT_RECORD_bSetFocus@@3PAU_jfieldID@@A 1000617c     Kernel32.obj
 0003:00000180       ?SMALL_RECT_Class@@3PAV_jclass@@A 10006180     Kernel32.obj
 0003:00000184       ?SMALL_RECT_Constructor@@3PAU_jmethodID@@A 10006184     Kernel32.obj
 0003:00000188       ?SMALL_RECT_Left@@3PAU_jfieldID@@A 10006188     Kernel32.obj
 0003:0000018c       ?SMALL_RECT_Top@@3PAU_jfieldID@@A 1000618c     Kernel32.obj
 0003:00000190       ?SMALL_RECT_Right@@3PAU_jfieldID@@A 10006190     Kernel32.obj
 0003:00000194       ?SMALL_RECT_Bottom@@3PAU_jfieldID@@A 10006194     Kernel32.obj
 0003:00000198       ?UnionChar_Class@@3PAV_jclass@@A 10006198     Kernel32.obj
 0003:0000019c       ?UnionChar_Constructor@@3PAU_jmethodID@@A 1000619c     Kernel32.obj
 0003:000001a0       ?UnionChar_UnicodeChar@@3PAU_jfieldID@@A 100061a0     Kernel32.obj
 0003:000001a4       ?__proc_attached@@3HA      100061a4     MSVCRT:dll_dllmain.obj
 0003:000001a8       _GS_ExceptionRecord        100061a8     MSVCRT:gs_report.obj
 0003:000001f8       _GS_ContextRecord          100061f8     MSVCRT:gs_report.obj
 0003:000004e8       ?is_initialized_as_dll@@3_NA 100064e8     MSVCRT:utility.obj
 0003:000004e9       ?module_local_atexit_table_initialized@@3_NA 100064e9     MSVCRT:utility.obj
 0003:000004ec       ?module_local_atexit_table@@3U_onexit_table_t@@A 100064ec     MSVCRT:utility.obj
 0003:000004f8       ?module_local_at_quick_exit_table@@3U_onexit_table_t@@A 100064f8     MSVCRT:utility.obj
 0004:00000060       $R000000                   10007060     le.dll.res
